:100000000C945B000C9483000C9483000C9483008C
:100010000C9483000C9483000C9483000C94830054
:100020000C9483000C9483000C9483000C94830044
:100030000C9483000C9483000C9483000C94830034
:100040000C940D030C9483000C9419050C948300FC
:100050000C9483000C9483000C9483000C94830014
:100060000C9483000C948300000024272A000025B0
:10007000282B000023262904040404040404040299
:100080000202020202030303030303010204081035
:100090002040800102040810200102040810200002
:1000A0000000070002010000030406000000000039
:1000B00000000000650111241FBECFEFD4E0DEBFB9
:1000C000CDBF11E0A0E0B1E0E4E8FBE002C00590A4
:1000D0000D92AE31B107D9F711E0AEE1B1E001C048
:1000E0001D92AC3BB107E1F710E0C6EBD0E004C0D5
:1000F0002297FE010E94BC05C43BD107C9F70E94AC
:100100005E010C94C0050C94000061E080910E012A
:100110000E94080480911401909115010E94A2038D
:1001200060E080910E010E94080480911601909178
:1001300017010E94A20360E071E08EE291E00E944C
:100140008E0160911401709115018EE291E00E9480
:10015000DD020E946A0360931E0170931F01809369
:1001600020019093210128EE33E040E050E00E940E
:100170006905C901DA018093220190932301A093BC
:100180002401B09325018A389105A105B105D1F16B
:100190008B389105A105B1055CF40097A105B10567
:1001A000C1F088389105A105B10509F058C01AC001
:1001B000883B9105A105B105A9F1883C9105A105F0
:1001C000B105E9F180399105A105B10509F047C0F4
:1001D0001CC061E080910C010E94080461E08091E4
:1001E000080108C060E0809108010E94080461E0F5
:1001F00080910C010E94080460E080910A010E9435
:1002000008042DC080E496E026C061E080910C01D6
:100210000E94080460E080910A010E94080487E9B6
:1002200093E019C061E080910C010E94080460E035
:1002300080910A010E94080480E699E00CC060E009
:1002400080910C010E94080461E080910A010E94E3
:10025000080482E796E09093150180931401409181
:1002600022015091230160912401709125018EE2B9
:1002700091E00E94CA02089540E855E260E070E013
:100280008EE291E00E94790161E0809108010E9474
:10029000EA0361E080910A010E94EA0361E0809133
:1002A0000C010E94EA0360E0809126010E94EA03AB
:1002B00061E080910E010E94EA0308950E94B0035C
:1002C0000E943C010E948500FDCF8CE191E090935B
:1002D0002F0180932E010895862F0E94D80408953F
:1002E0000E94100508950E94F10408950E94E00400
:1002F0000895CB01BA010E949F040895DC01ED919D
:10030000FC910190F081E02D09950895DC01ED91BB
:10031000FC910190F081E02D099508950F931F93B2
:10032000CF93DF938C01EB0109C02196D801ED91A9
:10033000FC910190F081E02DC80109956881662348
:10034000A1F7DF91CF911F910F9108950F931F9304
:100350008C01DC01ED91FC910190F081E02D6DE0CC
:100360000995D801ED91FC910190F081E02D6AE0B2
:10037000C80109951F910F9108950F931F938C0148
:10038000DC01ED91FC910190F081E02D0995C8010F
:100390000E94A6011F910F9108950F931F938C0146
:1003A0000E948E01C8010E94A6011F910F9108951D
:1003B0000F931F938C01DC01ED91FC910190F08172
:1003C000E02D0995C8010E94A6011F910F91089583
:1003D0002F923F924F925F926F927F928F929F9255
:1003E000AF92BF92CF92DF92EF92FF920F931F9343
:1003F000DF93CF93CDB7DEB7A0970FB6F894DEBFEB
:100400000FBECDBF1C016A017B014115510561057D
:10041000710549F4DC01ED91FC910190F081E02D32
:1004200060E3099554C0882499245401422E552430
:100430006624772401E010E00C0F1D1F080D191D24
:10044000C701B601A30192010E946905F80160830A
:100450000894811C911CA11CB11CC701B601A30109
:1004600092010E946905C901DA016C017D01C11484
:10047000D104E104F104F1F681E0E82EF12CEC0E58
:10048000FD1EE80CF91C3E010894611C711CD5018D
:10049000C4010197A109B1096C01C818D90814C099
:1004A000F601EE0DFF1D60816A3010F4605D01C041
:1004B000695CD101ED91FC910190F081E02DC101C9
:1004C00009950894E108F1086E147F0449F7A09695
:1004D0000FB6F894DEBF0FBECDBFCF91DF911F9155
:1004E0000F91FF90EF90DF90CF90BF90AF909F90D3
:1004F0008F907F906F905F904F903F902F900895D6
:100500002AE00E94E80108950F931F938C010E9436
:100510008002C8010E94A6011F910F910895AB01AE
:1005200060E070E00E94800208950F931F938C0199
:10053000AB0160E070E00E948002C8010E94A60149
:100540001F910F910895EF92FF920F931F93CF93F6
:10055000DF93EC017A018B0177FF0FC0E881F9810D
:100560000190F081E02D6DE2099510950095F094D1
:10057000E094E11CF11C011D111D2AE0B801A70146
:10058000CE010E94E801DF91CF911F910F91FF9062
:10059000EF9008950F931F938C010E94A302C8014E
:1005A0000E94A6011F910F910895AB01662757FD88
:1005B0006095762F0E94A30208950F931F938C01DC
:1005C000AB01662757FD6095762F0E94A302C801F4
:1005D0000E94A6011F910F910895DC01211531059C
:1005E00041F4ED91FC910190F081E02D642F09958B
:1005F00008952A30310519F40E94A30208950E943B
:10060000E80108950F931F938C010E94ED02C80129
:100610000E94A6011F910F9108951F920F920FB68D
:100620000F9211242F938F939F93AF93BF93809139
:10063000300190913101A0913201B091330180508D
:10064000904CAF4FBF4F8093300190933101A093F6
:100650003201B093330127C0809130019091310174
:10066000A0913201B091330180589E43A040B04028
:100670008093300190933101A0933201B093330104
:100680008091340190913501A0913601B0913701EC
:100690000196A11DB11D8093340190933501A09363
:1006A0003601B09337018091300190913101A091D2
:1006B0003201B091330181589E43A040B04060F6B2
:1006C000BF91AF919F918F912F910F900FBE0F907F
:1006D0001F9018958FB7F89420913401309135010F
:1006E00040913601509137018FBFB901CA01089579
:1006F000EF92FF920F931F937B018C018FB7F894B9
:10070000409134015091350160913601709137016B
:100710008FBF2FB7F8948091340190913501A0914B
:100720003601B09137012FBF841B950BA60BB70B79
:100730008E159F05A007B10760F31F910F91FF90E1
:10074000EF900895019759F0FC01EE0FFF1FEE0F97
:10075000FF1F32978FB7F8943197F1F78FBF089545
:10076000789484B5826084BD84B5816084BD85B58C
:10077000826085BD85B5816085BDEEE6F0E0808153
:1007800081608083E1E8F0E0808182608083808105
:1007900081608083E0E8F0E0808181608083E1EB2C
:1007A000F0E0808184608083E0EBF0E08081816014
:1007B0008083EAE7F0E080818460808380818260CA
:1007C00080838081816080838081806880831092B3
:1007D000C1000895282F30E0C90185579F4FFC01C3
:1007E000949129583F4FF9018491882381F0E82F93
:1007F000F0E0E859FF4FE491F0E0662329F48081AE
:1008000090958923808308958081892B8083089522
:10081000482F50E0CA0181569F4FFC012491CA0124
:1008200085579F4FFC01949149585F4FFA013491CD
:100830003323C1F1222331F1233021F48091800050
:100840008F7705C0243031F4809180008F7D8093B4
:10085000800018C0213019F484B58F7704C022308D
:1008600021F484B58F7D84BD0DC0263021F48091A4
:10087000B0008F7705C0273029F48091B0008F7DBC
:100880008093B000E32FF0E0E359FF4FE491F0E0F4
:10089000662329F48081909589238083089580813F
:1008A000892B80830895482F50E0CA0181569F4FBD
:1008B000FC012491CA0185579F4FFC01949149582E
:1008C0005F4FFA013491332319F420E030E035C052
:1008D000222331F1233021F4809180008F7705C0ED
:1008E000243031F4809180008F7D8093800018C087
:1008F000213019F484B58F7704C0223021F484B5F7
:100900008F7D84BD0DC0263021F48091B0008F779B
:1009100005C0273029F48091B0008F7D8093B0000E
:10092000E32FF0E0EE58FF4FE491F0E0808120E00B
:1009300030E0892311F021E030E0C9010895EF9201
:10094000FF920F931F937B018C0122E030E040E087
:1009500050E00E948B05205C3D4B404F5F4FCA0129
:10096000B901A80197010E948B05C901DA0101971D
:10097000A109B109292F3A2F4B2F552747FD5A9529
:100980000196A11DB11D2093C50081508093C40024
:10099000E1ECF0E0808180618083808188608083E9
:1009A0008081806880831F910F91FF90EF90089560
:1009B000982F8091C00085FFFCCF9093C6000895CA
:1009C000809138019091390180589F4F20913A01D0
:1009D00030913B01821B930B60E870E00E9456054A
:1009E000089540913A0150913B01809138019091D6
:1009F00039018417950719F42FEF3FEF0FC0FA0163
:100A0000E45CFE4F2081CA01019660E870E00E941C
:100A1000560590933B0180933A0130E0C901089557
:100A200080913A0190913B01909339018093380174
:100A300008951F920F920FB60F9211242F933F9398
:100A40004F935F936F937F938F939F93AF93BF93D6
:100A5000EF93FF934091C600E0913801F091390186
:100A6000CF01019660E870E00E9456059C018091DC
:100A70003A0190913B012817390739F0E45CFE4FA9
:100A800040833093390120933801FF91EF91BF915A
:100A9000AF919F918F917F916F915F914F913F9116
:100AA0002F910F900FBE0F901F90189597FB092E56
:100AB00007260AD077FD04D049D006D000201AF4CA
:100AC000709561957F4F0895F6F7909581959F4FAA
:100AD0000895A1E21A2EAA1BBB1BFD010DC0AA1F7F
:100AE000BB1FEE1FFF1FA217B307E407F50720F097
:100AF000A21BB30BE40BF50B661F771F881F991F12
:100B00001A9469F760957095809590959B01AC015A
:100B1000BD01CF01089597FB092E05260ED057FD84
:100B200004D0D7DF0AD0001C38F45095409530959A
:100B300021953F4F4F4F5F4F0895F6F79095809561
:100B4000709561957F4F8F4F9F4F0895AA1BBB1BD8
:100B500051E107C0AA1FBB1FA617B70710F0A61BBD
:100B6000B70B881F991F5A95A9F780959095BC01DE
:100B7000CD010895EE0FFF1F0590F491E02D09942B
:040B8000F894FFCF17
:100B84002050756C73653A000500080009000300E5
:0E0B94007807A0F640061400000000006C0177
:00000001FF
